:020000040000FA
:10040000052A000000000000090021009615852340
:100410001422AB232D22FD3308000800F000120047
:100420001E00F00BFC3308002100FC3099001A0973
:100430005139031DFC33270090309B008630850026
:10044000FF308400023087004030860007300E22E3
:100450004A233D008E018E1508003D0010184A2BDE
:10046000901D08000F088700901120007839031DA7
:10047000F33207199F322008343A031DA632452271
:100480002000B100090F6F328E32A001A401B01319
:10049000C01BB0174008C03A031957324108FB3E51
:1004A000031D0232B0160034090B2A32430B053209
:1004B00084308500E63084001234090B0532843024
:1004C0008500F83084006234090B12324230063C59
:1004D0000318FF34853085005A308400C20A043284
:1004E000003F84070318850AC20BFA33003F080057
:1004F000F43E031DFF3485308500E8308400393434
:100500000903090B0732FE303018FD3084008430B7
:1005100085000134090B0B324208B0000830452336
:10052000083038234830AC00BC00FB010034E93E01
:1005300003190232090B0632023085004030840074
:10054000FB010734090BFF340034410B05328630C0
:100550008500D33084002C34090BFF3486308500AD
:1005600021308400B2340508B3000408B200C70883
:10057000031D043231084602031CB1073D000E1270
:100580002000C01F093206234830012324094039C6
:100590000838A400A4170800A413A501B108031D7E
:1005A000F3330C30F2333D000E1220000C30C92220
:1005B0000C302732B01F02320623E833B01E080089
:1005C000B01242083D0096000800B01B1732B10877
:1005D0000319143233088500320884000030870084
:1005E00040308600A10803190532A10316001A0045
:1005F000B10BF8330508B3000408B20020094039F4
:100600000838A0001030A100A0170800A501B1080B
:100610000319080033088500320884000030870081
:1006200040308600251A053212001E00A50AB10BC3
:10063000F9330508B3000408B200080020002C09B3
:1006400040390838AC00AC17080020003C0940399C
:100650000838BC00BC170800071E0F32871D4A2C43
:10066000071D4B2C39080D22200038094039083865
:10067000B8004030A900B81708000719332C290822
:100680000C222000280940390838A8004030A90071
:10069000A81708003D00900114309100850120301A
:1006A0008400F00003011A00F00BFD333D000E172B
:1006B00096010E120E13901D033290112C22FB3363
:1006C000163098001E3099009B001A309A002000C6
:1006D0002030A3002030A2002030A7002030A60048
:1006E0002030AB003030AA002030AF007030AE00B8
:1006F0002130B7003030B6002030BB00B030BA0037
:100700002030BF00F030BE00D82A24000C12213067
:10071000950023008C018E0122008C018E011D1595
:10072000210013308C0006308E002C00063095001E
:10073000C030960020000B309B001C153130980013
:100740002400CC01E830CD00CE01CF00D001D10093
:10075000D201D30108002000111C0800111018104C
:10076000E53096074808973D1814F60AF61D08006C
:10077000F61121000E110C1222000E08083EF100A5
:100780003F398E00F83E090C1C39243E84000230AB
:1007900085000318850A24000430F000FF30910022
:1007A0002000911DFE339111240011081900F00B57
:1007B000F53321000C160E15711F08002400951248
:1007C00022000C1521000C112000BC1FF723200073
:1007D000FB08031903242400D20A0319D30A2100B9
:1007E0000E1522000C11240095162000080002307E
:1007F00085002030840020308700F03086002030D3
:10080000BD000E22252B24005208F2005308F300ED
:1008100020000A30F4008724FA01093055247A3583
:100820000935203E8600023087000318870A423FC0
:10083000F200433FF3006124FA0AFA1DEE330A3056
:1008400055240D3055244030AD007B02031CAD070C
:1008500002308500A0308400203087007030860090
:100860002D300E221E2B200040307B02AD00031CD9
:1008700007320130FB0002308500E0308400EC33A9
:10088000FB0124000830CC07031D0800E830CD0A26
:100890000319CD00080024000830CE07031D08000E
:1008A000E830CF0A0319CF000800F7007B08A03E0C
:1008B0008600023087000318870A77088100FB0A48
:1008C000080072183A327208F8000430F000F3376A
:1008D000F20CF00BFC330A30F4007E242E30552449
:1008E000F819043230307819323003323530781943
:1008F00037305524303078193530552CF31F0732F6
:100900002D305524F309F209F20A0319F30AF9010B
:10091000AA247908A32475088100F90A7308F2044F
:10092000031DF6337903A3240108F63E0318073E9E
:100930003A3E5524F90BF63308004E305524613009
:1009400055244E30552C473E860002308700031850
:10095000870A0800F5011030F000F235F30DF50DAF
:100960000318043274087502031C03327408F5027C
:100970007214F00BF23308008700230015140000F6
:10098000000013081A0014081A00910A0319920AA9
:10099000870BF43308002300151615150F322300BA
:1009A00095161515120093001200940011091F39B5
:1009B00003190332DE24910AF5339512553096005F
:1009C000AA3096009514000000000800123401348B
:1009D00010340234EF34023401341034D834043487
:1009E000DD34EF3411340034013402340334013483
:1009F0000934023462340034033401340034803466
:100A0000193409340434003400340234FF3400341F
:100A100000340534073405340334023440340034E0
:100A20000034073405348334023440340034003455
:100A300008340B34013402340234023400340434F8
:100A400009340434013400340134023402340134F2
:100A50000434053424340034103401340434243490
:100A600002340234053424340634003401340534AD
:100A7000243401340334013407340534823403341C
:100A800010340034023409340434023400340234A3
:100A90000A3400340034003407340534013402349D
:100AA0004034003400340734053481340234403497
:100AB000003400340434033407340434223403345F
:100AC000543400345534003420340034433400347A
:100AD00068340034653400346D3400346E340034CE
:100AE00069340034743400347A3400342C340034E3
:100AF0002034003445340034573400344134003459
:100B00002234033438340034203400345434003474
:100B10006834003465340034723400346D34003489
:100B20006F340034653400346C3400346534003480
:100B30006D340034653400346E3400347434003461
:100B400065340034303403346834003465340034A0
:100B50006834003461340034403400346834003484
:100B6000723400347A3400342E3400347434003457
:100B7000753400342D340034633400346834003468
:100B8000653400346D3400346E340034693400341C
:100B9000743400347A3400342E3400346434003435
:100BA00065340034083403344334003444340034AE
:100BB000433400340E340334573400346534003485
:100BC0006234003455340034533400344234003439
:100BD00005340F34393400340234183410340534F9
:100BE00000343834B63408343434A9340934A034E9
:100BF00047348B34FD34A034763488341534B6341D
:100C0000653400340134013401341C3410340534AB
:100C10000034DF346034DD34D83489344534C734AB
:100C20004C349C34D23465349D349E3464348A34DC
:100C30009F340034003403340634B23400340234B8
:100C400000340A34003400340034003400340334F7
:100C50000634B23400340834003401340034003433
:100C60000034A83400340834003402340034003432
:100C70000034A034003414340034033400345734C6
:100C800049344E3455345334423400340034003443
:100C90000034003400340034003400340034843430
:100CA000003404340034073400342A34003444342B
:100CB00000346534003476340034693400346334ED
:100CC000003465340034493400346E3400347434F4
:100CD00000346534003472340034663400346134D6
:100CE0000034633400346534003447340034553400
:100CF0000034493400344434003473340034003454
:100D00000034503400347B34003439340034373408
:100D10000034353400344634003434340034343450
:100D2000003444340034393400342D340034303449
:100D300000344434003430340034383400342D343A
:100D40000034343400343334003446340034443412
:100D500000342D3400343834003442340034333419
:100D60000034453400342D3400343134003432340E
:100D700000343734003443340034413400343834E0
:100D800000344134003446340034463400344634B0
:100D9000003439340034443400347D3400340034B9
:100DA0000034003400342C34033401347734773485
:100DB00077342E34743475342D34633468346534A8
:100DC0006D346E34693474347A342E34643465345A
:100DD0002F347E3468346534683461342F3465349C
:100DE000773461342F344F34663465346E342F34A5
:100DF0003834743465342E34683474346D3480344B
:0C0E000025340034003400340034083481
:00000001FF
